:1000000093C00000ADC00000ABC00000A9C000005C
:10001000A7C00000A5C00000A3C00000A1C0000050
:100020009FC000009DC000009BC000000C94F10F19
:1000300097C0000095C0000093C000000C94AF0A68
:100040008FC000008DC000008BC0000089C0000080
:1000500087C0000085C0000083C0000081C0000090
:100060007FC000007DC000007BC0000079C00000A0
:1000700077C0000012011001FF000010EB03042103
:1000800000020102030109022000010100C032093F
:1000900004000002FF000000070582024000000784
:1000A000050202400000040309041803440065002F
:1000B00061006E002000430061006D006500720069
:1000C0006100000044034C00550046004100200040
:1000D00041005600520049005300500020004D00DE
:1000E0006B0049004900200043006C006F006E0067
:1000F00065002000500072006F0067007200610010
:100100006D006D006500720000001C0330003000BF
:100110003000300041003000300031003200380043
:10012000320035003500000011241FBECFEFD2E0B1
:10013000DEBFCDBF11E0A0E0B1E0EAEAF1E202C02B
:1001400005900D92AC33B107D9F711E0ACE3B1E003
:1001500001C01D92A535B107E1F756D00C94D3101C
:100160004FCF85B18F70806685B9089585B18F7046
:10017000806185B9089580914C01843081F482E0DA
:100180008093E9008091E80082FF09C085B18F70FB
:10019000806385B978D085B18F70806A85B90895FC
:1001A00085B18F70806A85B982E060E842E30E9481
:1001B000350E882321F485B18F70806585B9089547
:1001C00084B7877F84BF88E10FB6F894809360007E
:1001D000109260000FBE80E090E020E80FB6F89427
:1001E00020936100809361000FBE84B1806F84B959
:1001F00085B18F7085B90E94E40F8AEF87BD82E0D8
:1002000084BD83E085BD0895DBDF87D185B18F7024
:10021000806185B9B0DF44D10E949810FBCFDA012C
:10022000923049F0933061F0913029F5E4E7F0E045
:1002300022E130E024C0E6E8F0E020E230E01FC038
:10024000813059F0813028F0823059F0833099F4B0
:100250000CC0E6EAF0E084910BC0EAEAF0E0849199
:1002600007C0E4ECF0E0849103C0EAE0F1E084919F
:10027000282F30E004C0E0E0F0E020E030E0ED9333
:10028000FC93C9010895FF920F931F931091F10001
:10029000143109F4BEC0153110F51A3009F49FC0AD
:1002A0001B3068F4143038F4123008F053C01130A9
:1002B00009F0CBC033C0163009F0C7C078C0113187
:1002C00009F4A2C0123120F4103109F0BEC09AC066
:1002D000123109F4A1C0133109F0B7C097C0193128
:1002E00009F49FC01A3168F4163109F492C016312E
:1002F00008F48CC0173109F494C0183109F0A5C076
:100300008DC01D3109F490C01D3108F487C010352F
:1003100009F48EC0113509F098C088C08091E800BA
:10032000982F9B7F9093E8008F778093E8008091CF
:10033000EC0081608093EC001093F1001092F100CA
:100340008AE08093F10080E091E06AE070E00E9432
:10035000B30E92C00091F100123011F0FF2402C0E0
:10036000F090F1008091E800982F9B7F9093E80037
:100370008F778093E8008091EC0081608093EC009F
:100380001093F100802FAED0123041F481FF0DC0E8
:100390001092F100802F6F2DADD06EC080FF05C090
:1003A0001092F100802F96D065C080EC63C08DE381
:1003B00091E064E070E00E94150F8091E800982FB2
:1003C0009B7F9093E8008F778093E8008091EC000A
:1003D00081608093EC0081E080933C010EC08091AD
:1003E000E800982F9B7F9093E8008F778093E80038
:1003F0008091EC0081608093EC001093F1001092EA
:10040000F1003AC071D441C033D43FC0812FBAD279
:100410003CC0812FF5D139C0AAD137C0812F55D129
:1004200034C0812F0CD131C092D02FC0A2D52DC0A5
:100430000CD72BC08091E800982F9B7F9093E80009
:100440008F778093E8000E94880E8091F2008034BC
:1004500089F38091E800982F9B7F9093E8008F7735
:100460008093E8008091EC0081608093EC00109311
:10047000F10089EC8093F1008091E800982F9E7F35
:100480009093E8008F778093E8000E94880E809117
:10049000EC008E7F8093EC001F910F91FF900895E8
:1004A0000895282FEBE0F1E090E08081281751F4C7
:1004B000892F90E063E070E00E94AB109C01255F03
:1004C0003E4F06C09F5F33969A3079F720E030E0C8
:1004D000C9010895E6DFFC01009711F480E008955A
:1004E00081810895DEDFFC01009711F480E008951A
:1004F000828108950F931F93182F062FD2DFFC01DE
:10050000009741F001831E3929F480E090E0602FCC
:100510000E94C5101F910F9108950F931F938EE9AC
:10052000C0DF8C0180E090E00E94BD10F801818363
:100530001F910F910895982F16BC82E085BB04C0CF
:10054000A99BFECF85BB91509923D1F708950F93B6
:100550001F93DF93CF93CDB7DEB7C250D1400FB614
:10056000F894DEBF0FBECDBFCE01019663E070E010
:100570000E94E40E8E010C5F1F4F6981C80170E07C
:100580000E94E40E8091E800982F9B7F9093E800F2
:100590008F778093E8008091EC0081608093EC007D
:1005A0008DE18093F1001092F1002B81698190E040
:1005B000A80110C0961748F4FA01E90FF11D8081D7
:1005C0008EBD0DB407FEFDCF04C01EBC0DB407FEEA
:1005D000FDCF9F5F921770F33A8190E0AE014C5FC0
:1005E0005F4F14C0261750F4FA01E20FF11D80810D
:1005F0008EBD0DB407FEFDCF2F5F04C01EBC0DB431
:1006000007FEFDCF8EB58093F1009F5F931750F3E7
:100610001092F1008091E800982F9E7F9093E8005F
:100620008F778093E800CE5FDE4F0FB6F894DEBF81
:100630000FBECDBFCF91DF911F910F910895FF9213
:100640000F931F93DF93CF9300D000D0CDB7DEB7C9
:10065000F82E8E010F5F1F4FC80164E070E00E940A
:10066000E40E8091E800982F9B7F9093E8008F77AD
:100670008093E8008091EC0081608093EC00F801A9
:100680009E012B5F3F4F80818EBD0DB407FEFDCFD5
:100690003196E217F307B9F7F092F1001092F100EA
:1006A0001092F1008091E800982F9E7F9093E800CF
:1006B0008F778093E8000F900F900F900F90CF915D
:1006C000DF911F910F91FF9008951F93DF93CF93B8
:1006D000CDB7DEB729970FB6F894DEBF0FBECDBFFA
:1006E000182FCE01059665E070E00E94E40E80911F
:1006F000E800982F9B7F9093E8008F778093E80025
:100700008091EC0081608093EC00FE013696DE0162
:1007100011969E01265F3F4F80818EBD0DB407FE6E
:10072000FDCF8EB58D933196E217F307A9F710939D
:10073000F1001092F1008D81FE01E80FF11D808122
:100740008093F1001092F1008091E800982F9E7F35
:100750009093E8008F778093E80029960FB6F8947D
:10076000DEBF0FBECDBFCF91DF911F910895DF9304
:10077000CF9300D000D000D0CDB7DEB7CE01019628
:1007800066E070E00E94E40E8091E800982F9B7F65
:100790009093E8008F778093E8008091EC0081606F
:1007A0008093EC00FE0133969E01295F3F4F8081CC
:1007B0008EBD0DB407FEFDCF3196E217F307B9F7F2
:1007C0008A81882321F48981B6DE90E002C034D387
:1007D000982F82E18093F1009093F1008091E800DE
:1007E000982F9E7F9093E8008F778093E80026965D
:1007F0000FB6F894DEBF0FBECDBFCF91DF91089545
:10080000EF92FF920F931F93DF93CF9300D00F923D
:10081000CDB7DEB7F82ECE01019663E070E00E94FE
:10082000E40E99818A8189839A838091E800982FC8
:100830009B7F9093E8008F778093E8008091EC0095
:1008400081608093EC00F092F1001092F1008091B1
:100850003C01882369F080913D0190913E01A09177
:100860003F01B0914001B7FF01C058D310923C0145
:1008700000E010E05BC0C80181709070E82E882312
:1008800031F084E1F81619F48B81886002C08B8105
:10089000877F8B838B818EBD0DB407FEFDCF2091AA
:1008A0003D0130913E0140913F0150914001BB27F5
:1008B000A52F942F832F8EBD0DB407FEFDCF2EBD27
:1008C0000DB407FEFDCF1EBC0DB407FEFDCF8EB5E7
:1008D0008093F1008091E80085FD0BC08091E800D5
:1008E000982F9E7F9093E8008F778093E8000E9476
:1008F000880EEE2019F084E1F81619F086E1F8165A
:1009000099F480913D0190913E01A0913F01B091F9
:1009100040010196A11DB11D80933D0190933E01C0
:10092000A0933F01B09340010F5F1F4F89819A81CF
:100930000817190708F49FCF1092F1008091E80082
:100940009091E800292F2E7F2093E8009F779093C5
:10095000E80085FD0DC00E94880E8091E800982F68
:100960009E7F9093E8008F778093E8000E94880E26
:100970000F900F900F90CF91DF911F910F91FF90EB
:10098000EF9008955F926F927F928F929F92AF92B5
:10099000BF92CF92DF92EF92FF920F931F93DF935C
:1009A000CF93CDB7DEB7C950D1400FB6F894DEBFB4
:1009B0000FBECDBFB82ECE01019669E070E00E9457
:1009C000E40E79816A8181E06130780790F080914E
:1009D000E800982F9B7F9093E8008F778093E80042
:1009E0008091EC0081608093EC00B092F10080EC8B
:1009F0001DC17A836983CE010A960E94E40E80911C
:100A0000E800982F9B7F9093E8008F778093E80011
:100A10008091EC0081608093EC00A3E1BA1611F4A0
:100A2000A88401C0A98480913C01882369F0809149
:100A30003D0190913E01A0913F01B0914001B7FF6F
:100A400001C06CD210923C01FB80BE01665F7F4FFB
:100A5000F0FC06C06B01EE24FF2488249924DDC03D
:100A600050903D0190903E0169807A80ED80CF806A
:100A7000252D392D40913F0150914001C901DA01E6
:100A80009C01AD01E0E0F0E000E010E03DC0CF01EE
:100A900081709070882EDB01DC90882331F0B3E107
:100AA000BB1619F488E0E82A02C0A7EFEA22EEBCE0
:100AB0000DB407FEFDCFBB27A52F942F832F8EBD2E
:100AC0000DB407FEFDCF2EBD0DB407FEFDCFDEBC7D
:100AD0000DB407FEFDCF0115110551F4DA1441F0F4
:100AE000882029F0B3E1BB1611F488E0C82A8901F7
:100AF000882019F4A5E1BA1621F42F5F3F4F4F4F1C
:100B00005F4F6F5F7F4F3196E615F70508F4BFCF53
:100B1000ED82CF8220933D0130933E0140933F010F
:100B200050934001F7FE7FC08E818EBD0DB407FE4D
:100B3000FDCF852D9EBC0DB407FEFDCF8EBD0DB43F
:100B400007FEFDCF1EBC0DB407FEFDCF011511053C
:100B500029F4BFEDFB22E0E1FE2AFB828B81B80184
:100B60004A2D2C810C2D8ED15FC0C70181709070F1
:100B7000782FD6016C91882331F0B4E1BB1619F4BB
:100B80008D81886002C08D81877F8D838D818EBD30
:100B90000DB407FEFDCF20913D0130913E01409103
:100BA0003F0150914001BB27A52F942F832F8EBD6D
:100BB0000DB407FEFDCF2EBD0DB407FEFDCF6EBDFB
:100BC0000DB407FEFDCF6A1549F0772331F0E3E15C
:100BD000BE1619F48F8188608F834901772319F439
:100BE000F5E1BF1661F42F5F3F4F4F4F5F4F2093EA
:100BF0003D0130933E0140933F01509340018B8172
:100C0000B4014A2D2C810F813DD1882369F40894C9
:100C1000C11CD11C0894E11CF11C89819A81E81641
:100C2000F90608F4A2CF80E0B092F1008093F100C1
:100C30008091E800982F9E7F9093E8008F778093B3
:100C4000E800C75FDE4F0FB6F894DEBF0FBECDBF22
:100C5000CF91DF911F910F91FF90EF90DF90CF9098
:100C6000BF90AF909F908F907F906F905F9008950E
:100C70000F931F93DF93CF9300D0CDB7DEB7CE0194
:100C8000019662E070E00E94E40E08EE10E0F801C8
:100C90008081982F9B7F90838F778083ECEEF0E0AC
:100CA000808181608083898146DC80E04BD184B182
:100CB000897F84B985B1867F85B91CBC1DBC8A81BA
:100CC0003ADCE1EFF0E081E180831082F80180817D
:100CD000982F9E7F90838F7780830F900F90CF9176
:100CE000DF911F910F9108956F927F928F929F9243
:100CF000AF92BF92DF92EF92FF920F931F93DF9319
:100D0000CF93CDB7DEB72F970FB6F894DEBF0FBEE7
:100D1000CDBFCE0105966BE070E00E94E40E80919D
:100D2000E800982F9B7F9093E8008F778093E800EE
:100D30008091EC0081608093EC0010923D01109254
:100D40003E0110923F01109240018F81F4DB06D1E9
:100D5000282F206194B1966094B995B1996095B9A6
:100D600080658CBD26FF03C08DB5816002C08DB546
:100D70008E7F8DBD00ECD02E1CE0612E712C6C0E90
:100D80007D1E4E010894811C911CB0E1AB2EB12C4C
:100D9000AC0EBD1E29C08150888781E0D3D08E81E2
:100DA000CADB830174018985C6DBF80180818EBDB1
:100DB0000DB407FEFDCF8EB5F70181937F010F5F64
:100DC0001F4F0A151B0579F78B85882361F0FE01FB
:100DD000E80FF11D90818A85981729F080E0B2D044
:100DE0008E81A9DB01C0DD248885882319F0F0EC11
:100DF000DF1689F280E18093F100D092F1008091BA
:100E0000E800982F9E7F9093E8008F778093E8000A
:100E10002F960FB6F894DEBF0FBECDBFCF91DF91F6
:100E20001F910F91FF90EF90DF90BF90AF909F9038
:100E30008F907F906F90089516BC82E085BB80EF05
:100E400020EF92E02EBD0DB407FEFDCF1EBC0DB409
:100E500007FEFDCF1EBC0DB407FEFDCFA99B02C04F
:100E600095BB81501EBC0DB407FEFDCF0EB400FE35
:100E700003C0882339F704C0882311F080E0089567
:100E800081E808950F9390E08E778830910509F4FA
:100E90003EC08930910534F48230910559F00497B1
:100EA000C1F513C08032910581F08034910579F14C
:100EB000409779F516BC82E085BB04C0A99BFECFA4
:100EC00085BB21502223D1F724C016BC82E085BB0C
:100ED00090EF22E00EBD0DB407FEFDCF7EBD0DB438
:100EE00007FEFDCF6EBD0DB407FEFDCFA99B02C06E
:100EF00025BB91501EBC0DB407FEFDCF8EB58417E7
:100F000019F0992339F707C0992319F404C094DF25
:100F100003C080E001C080E80F9108958DE48EBD8C
:100F20000DB407FEFDCF1EBC0DB407FEFDCF8091B2
:100F30003F018EBD0DB407FEFDCF1EBC0DB407FEF4
:100F4000FDCF0895882339F03E9A8EE9C3DA8823CD
:100F500021F4469A08953E984698089588E9BADAA9
:100F6000873008F086E0E82FF0E0E75DFE4F8081F3
:100F70000895DF93CF930F92CDB7DEB7CE010196E0
:100F800061E070E021D78091E800982F9B7F9093DB
:100F9000E8008F778093E8008091EC008160809377
:100FA000EC0081E58093F1008981882311F080ECC9
:100FB00001C080E08093F1008091E800982F9E7F2F
:100FC0009093E8008F778093E8000F90CF91DF91A6
:100FD0000895AF92BF92CF92DF92EF92FF920F935C
:100FE0001F93DF93CF93CDB7DEB7C850D1400FB674
:100FF000F894DEBF0FBECDBFCE01019668E070E071
:10100000E3D62B813C814D815E81122F0027FF2486
:10101000EE24852F9927AA27BB27E82AF92A0A2B2D
:101020001B2BDA01C90180709070B070892F9A2F44
:10103000AB2FBB27E82AF92A0A2B1B2B2070407004
:101040005070542F432F322F2227E22AF32A042BE9
:10105000152BEB82FC820D831E837F8168856F8355
:101060007887CE010996B0D68091E800982F9B7FB3
:101070009093E8008F778093E8008091EC00816086
:101080008093EC008981813011F444E217C08230F2
:1010900011F44CE213C0833021F444E383E366E3AC
:1010A0000FC0863021F483E08A834AE107C0843090
:1010B00011F48CE43BC08530C1F14EE283E266E27C
:1010C000EB80FC800D811E81AF80B8842A8199E07D
:1010D000C92ED12CCC0EDD1E73D3882311F090E0E5
:1010E00001C093E080E58093F10084E08093F100FB
:1010F0009093F1008091E800982F9E7F9093E800F4
:101100008F778093E800C85FDE4F0FB6F894DEBF9C
:101110000FBECDBFCF91DF911F910F91FF90EF9048
:10112000DF90CF90BF90AF90089588E04B815C81B5
:101130006D817E819E01275F3F4FAED3CECFEF9270
:10114000FF920F931F93DF93CF93CDB7DEB7C750B6
:10115000D1400FB6F894DEBF0FBECDBFCE010196D1
:1011600067E070E031D6EA80FB800C811D819E2D06
:10117000882777276627212F332744275527622B77
:10118000732B842B952BA801970120703070507021
:10119000232F342F452F5527622B732B842B952B10
:1011A00020E03FEF40E050E0E222F3220423152349
:1011B000102F0F2DFE2CEE246E297F29802B912BD2
:1011C0006A837B838C839D833E812F812E833F8323
:1011D0004091E800542F5B7F5093E8004F77409395
:1011E000E8004091EC0041604093EC00AE01485FA4
:1011F0005F4F76D3882311F493E001C090E080E53F
:101200008093F10085E08093F1009093F1009923A1
:1012100029F46E817F81CE010896A5D58091E800E2
:10122000982F9E7F9093E8008F778093E800C95FA6
:10123000DE4F0FB6F894DEBF0FBECDBFCF91DF916A
:101240001F910F91FF90EF900895CF92DF92EF9250
:10125000FF920F931F93DF93CF93CDB7DEB76297C3
:101260000FB6F894DEBF0FBECDBF1091F100143061
:1012700009F4DAC0153050F4123009F44CC01330C0
:1012800008F064C0113009F05BC10AC0163009F4DF
:10129000CFC0163008F4CAC0173009F051C107C1D9
:1012A0008091E800982F9B7F9093E8008F77809340
:1012B000E8008091EC0081608093EC00E6D181EC45
:1012C00097D189E595D180EE93D18E010E5E1F4FA7
:1012D000BBE0CB2ED12CCC0EDD1EAAE0EA2EF12CE9
:1012E000EC0EFD1ED601E4E3F1E088E001900D92E2
:1012F0008150E1F7F80180817BD1015010400E153B
:101300001F0581F7D5D190E59093F10091E090937E
:10131000F1009827C9C08091E800982F9B7F909397
:10132000E8008F778093E8008091EC0081608093E3
:10133000EC0081EC5DD180E05BD154D180E58093FD
:10134000F1001093F1001092F100F1C0CE01069669
:1013500065E070E039D52F81388549855A85122F8F
:101360000027FF24EE24852F9927AA27BB27E82AE8
:10137000F92A0A2B1B2BDA01C90180709070B0701A
:10138000892F9A2FAB2FBB27E82AF92A0A2B1B2B70
:10139000207040705070542F432F322F2227E22AA2
:1013A000F32A042B152B8091E800982F9B7F9093B4
:1013B000E8008F778093E8008091EC008160809353
:1013C000EC008E81813011F480E41DC0823011F474
:1013D00080E219C0833011F488E615C0843011F41E
:1013E00080E311C0853011F482E20DC0863011F423
:1013F0008AE209C0873011F482E305C0883011F415
:1014000088E101C080E0EF82F88609871A87B80179
:10141000A701ACD1882311F493E001C090E080E5EE
:101420008093F10083E03EC0D4DD8AC088DE88C0AE
:10143000CE01019661E070E0C7D48091E800982F5A
:101440009B7F9093E8008F778093E8008091EC0079
:1014500081608093EC008981813011F488E305C0BC
:10146000823011F088E701C089E3BE016E5F7F4FD3
:1014700071D2882311F493E001C090E080E580935D
:10148000F10086E08093F1009093F100992309F038
:101490004EC08A819B81AC81BD819D014427552727
:1014A0002093F1008093F1009093F10040C080916F
:1014B000F100813089F43091F1002091F100909198
:1014C000F1008091F10080933001909331012093DD
:1014D00032013093330114C0823011F021E011C089
:1014E0008091F100382F8091F100282F40E050E0EA
:1014F00020934101309342014093430150934401B2
:1015000020E08091E800982F9B7F9093E8008F77F0
:101510008093E8008091EC0081608093EC0080E58E
:101520008093F10087E08093F1002093F100809197
:10153000E800982F9E7F9093E8008F778093E800D3
:1015400062960FB6F894DEBF0FBECDBFCF91DF918C
:101550001F910F91FF90EF90DF90CF9008951F9211
:101560000F920FB60F9211248F939F93369A8BB5DB
:10157000882389F1469B15C080914701882359F53E
:101580008BB58C3011F41B9926C01B9B17C0809122
:1015900045019091460198609093460180934501E2
:1015A0000DC0809147018823B1F080914501909151
:1015B000460180FF02C02B9A01C02B988091450103
:1015C00090914601969587959093460180934501A9
:1015D0008BB581508BBD9F918F910F900FBE0F9057
:1015E0001F90189523983E982B98469815BC0895FF
:1015F000982F80914701882329F42B9A239A81E020
:1016000080934701292F30E0220F331F3C6040E0D8
:1016100052E005C024273527892F8150982399232C
:10162000C9F78BB58823E9F730934601209345012C
:101630008CE08BBD089580914701882339F08BB5EC
:101640008823E9F723982B98109247018CE08BBDF3
:101650008BB58823E9F78091450190914601089563
:1016600080914701882329F42B9A239A81E0809363
:1016700047018BB58823E9F78FEF9FE090934601F0
:10168000809345018CE08BBD0895239A3E9A2B9A56
:101690000000000080E590E090938900809388002E
:1016A00089E08093810082E080936F00D9DFD8CFFA
:1016B0000F931F9316BC82E085BB18EC02E080E814
:1016C00097DFB9DF81FF02C081E006C0A99BF7CF99
:1016D00005BB1150A1F780E01F910F910895EF9283
:1016E000FF920F931F937B018C01862F81DFBB2715
:1016F000A12F902F8F2D7CDFC801AA27BB2778DF71
:10170000E12EFF24002711278E2D72DF1F910F91EC
:10171000FF90EF90089590E0A0E0B0E020913001BC
:10172000309131014091320150913301822B932B42
:10173000A42BB52BBC01CD01D2CF0F931F9316BCA8
:1017400082E085BB18EC02E08CE052DF8FE0E3DF43
:1017500072DF87FD02C081E006C0A99BF5CF05BB03
:10176000115091F780E01F910F910895DF92EF9251
:10177000FF920F931F93D82E7A018B01DEDF88230F
:10178000C9F08CE435DF8AE0C6DF8D2D31DF80E4DF
:10179000D81631F48CE42CDF8BE0BDDF81E006C08D
:1017A0008CE426DFC801B7019ADF80E021DF80DF0B
:1017B000811181E01F910F91FF90EF90DF900895CC
:1017C0006F927F928F929F92AF92BF92CF92DF9251
:1017D000EF92FF920F931F93CF93DF93782E962E65
:1017E000642E822E20FF10C0A8DF882309F444C095
:1017F0008CE4FEDE8AE08FDF892DFADE8CE4F8DEF1
:101800008BE089DF81E0F4DEA114B10409F195DFFA
:10181000882309F431C08CE4EBDE8AE07CDF872D7D
:10182000E7DE8BE6E5DEC801B70159DF80EAE0DEDE
:101830008A2D8150DDDE84E6DBDEC0E0D0E005C02D
:10184000F60181916F01D4DE2196CA15DB05C0F344
:1018500081FE10C072DF882379F08CE4C9DE8AE053
:101860005ADF862DC5DE8CE4C3DEC801B70137DF41
:1018700080E0BEDE81E001C080E0DF91CF911F916A
:101880000F91FF90EF90DF90CF90BF90AF909F901F
:101890008F907F906F900895DF92EF92FF920F9359
:1018A0001F93CF93DF93D82E7A018B01E90145DF97
:1018B000882371F08CE49CDE8AE02DDF8D2D98DE8C
:1018C0008CE496DEC801B7010ADF888191DE81E0F1
:1018D000DF91CF911F910F91FF90EF90DF900895CE
:1018E000AF92BF92CF92DF92EF92FF920F931F932E
:1018F000CF93DF937B018C015A0169011EDF88239E
:10190000F1F08CE475DE8AE006DF83E471DE8BE6BD
:101910006FDEC801B701E3DE80EA6ADE8C2D8150FC
:1019200067DE84E265DEC0E0D0E005C084DEF5015C
:1019300081935F012196CC15DD05C0F381E0DF9135
:10194000CF911F910F91FF90EF90DF90CF90BF90BC
:10195000AF900895EF92FF920F931F93CF93DF9371
:10196000E82EEB01EADE882309F452C08CE440DE65
:101970008AE0D1DE8E2D3CDE8CE43ADE8BE0CBDEDD
:1019800081E036DE95DE882309F442C0D6DE882366
:1019900009F43EC0188219821A821B828CE028DE6C
:1019A00084E0B9DE48DE90E0A0E0B0E0888399836F
:1019B000AA83BB838CE01CDE85E0ADDEE880F98085
:1019C0000A811B8138DE382F20E040E050E02E29CC
:1019D0003F29402B512B288339834A835B838CE03A
:1019E00007DE86E098DEE880F9800A811B8123DE2D
:1019F00090E0A0E0B0E0DC01992788278E299F299C
:101A0000A02BB12B88839983AA83BB8381E001C07B
:101A100080E0DF91CF911F910F91FF90EF9008959B
:101A20001F93DF93CF9300D0CDB7DEB7EDE4F1E0A5
:101A30008091F100819381E0E535F807C9F7809145
:101A40004D0130914E01353009F486C0363040F4F6
:101A50003130C1F1313070F0333009F0F1C032C0B3
:101A6000383009F4BDC0393009F4D0C0363009F03F
:101A7000E7C091C0803821F0823809F0E1C008C089
:101A80009091480180914901882391F0926010C0A3
:101A9000809151018093E9008091EB0090E025E076
:101AA000969587952A95E1F7982F91701092E90005
:101AB0008091E800877F8093E8009093F100109276
:101AC000F10099C0882319F0823009F0B9C090E084
:101AD0008F719070009721F0029709F0B2C00CC08E
:101AE00080914F01813009F0ACC010924901333030
:101AF00069F5809349012AC080914F01882331F50F
:101B000020915101277009F49CC02093E900809135
:101B1000EB0080FF1BC0333021F48091EB0080622A
:101B200013C08091EB0080618093EB0081E090E036
:101B300002C0880F991F2A95E2F78093EA0010925D
:101B4000EA008091EB0088608093EB001092E9003E
:101B50008091E800877F56C0882309F071C01091FA
:101B60004F018091E800877F8093E800A8D005C0EE
:101B700080914C01882309F464C08091E80080FFC3
:101B8000F7CF912F9F7719F083E080934C019068F5
:101B90009093E30056C08058823008F051C0809185
:101BA0004F019091500160915101AE014F5F5F4F25
:101BB0000E940F01BC01009709F443C08091E80026
:101BC000877F8093E80089819A8160D18091E800C5
:101BD000982F9B7F9093E8008F778093E80031C027
:101BE000803871F58091E800877F8093E8008091CC
:101BF0004A018093F1008091E800982F9E7F909396
:101C0000E8008F778093E8005AD01BC08823C1F486
:101C100090914F019230A8F48091E800877F8093E3
:101C2000E80090934A014BD080914A01882311F437
:101C300083E001C084E080934C010E94D00001C089
:101C4000C9D18091E80083FF0AC08091EB008062D7
:101C50008093EB008091E800877F8093E8000F90ED
:101C60000F90CF91DF911F9108958093E9008091AB
:101C7000EB0081608093EB001092ED006093EC002C
:101C80004093ED008091EE00881F8827881F0895FB
:101C90001092F40090E09093E9001092F0001092FE
:101CA000E8008091ED008D7F8093ED008091EB0046
:101CB0008E7F8093EB009F5F953069F70895809148
:101CC0004D018823BCF404C080914C018823F9F0B5
:101CD0008091E80082FFF8CF8091E800982F9B7FE9
:101CE0009093E8008F778093E800089580914C01ED
:101CF000882369F08091E80080FFF8CF8091E800A8
:101D0000982F9E7F9093E8008F778093E800089546
:101D100094E68091EC0080FF05C08091E80080FF90
:101D200005C01FC08091E80082FD1BC080914C015E
:101D3000882311F482E008958091EB0085FF02C0B2
:101D400081E008958091E10082FFE3CF8091E1007E
:101D50008B7F8093E100992311F483E008959150E3
:101D6000D8CF80E00895FF920F931F93CF93DF9316
:101D7000182F092FEB01CCDFF82E8823F1F4812FE7
:101D8000902F9C01890117C08091E80085FD0DC04E
:101D90008091E800982F9E7F9093E8008F77809342
:101DA000E800B6DF882339F009C0F80181918F017E
:101DB0008093F1002197209739F78F2DDF91CF91F4
:101DC0001F910F91FF900895FF920F931F93CF9350
:101DD000DF93182F092FEB019BDFF82E8823F1F4F6
:101DE000812F902F9C01890117C08091E80085FD0B
:101DF0000DC08091E800982F9B7F9093E8008F772B
:101E00008093E80085DF882339F009C08091F100D4
:101E1000F80181938F012197209739F78F2DDF915A
:101E2000CF911F910F91FF900895FF920F931F93F1
:101E3000CF93DF938C01EB016BDFF82E8823F9F44D
:101E400021970C0F1D1F219618C08091E80085FD79
:101E50000DC08091E800982F9B7F9093E8008F77CA
:101E60008093E80055DF882341F00AC08091F1009B
:101E7000F8018083015010402197209731F78F2D72
:101E8000DF91CF911F910F91FF9008959C01409198
:101E90005301509154014617570710F460E043C0B6
:101EA0006115710511F0AB01F9CF8091E800982F11
:101EB0009E7F9093E8008F778093E80040E050E0A9
:101EC000EDCF8091E80083FF02C081E0089580910A
:101ED000E80082FD32C080914C018823A1F18091FD
:101EE000E80080FF20C08091F20090E009C0F90175
:101EF0002F5F3F4FE491E093F10041505040019635
:101F00004115510519F08031910588F360E0409743
:101F100009F461E08091E800982F9E7F9093E8009B
:101F20008F778093E8004115510559F6662349F6ED
:101F300004C080914C01882331F08091E80082FF39
:101F4000F8CF80E0089582E0089545D047D0109200
:101F50004C0110924A01109249011092480184E00C
:101F600089BD89B5826089BD09B400FEFDCF80912D
:101F7000D800982F9F779093D80080688093D800DE
:101F8000809163008E7F809363008091D8008F7D65
:101F90008093D8008091E0008E7F8093E000809154
:101FA000E1008E7F8093E1008091E2008160809368
:101FB000E2008091E100877F8093E1008091E20060
:101FC00088608093E2000895C0DF81E080934B0138
:101FD0007894089508951092E20008951092E10017
:101FE00008951F920F920FB60F9211242F933F93D3
:101FF0004F935F936F937F938F939F93AF93BF9311
:10200000EF93FF938091E10080FF1DC08091E2007B
:1020100080FF19C08091E1008E7F8093E100809164
:10202000E2008E7F8093E2008091E20080618093E5
:10203000E2008091D80080628093D80019BC109291
:102040004C010E94B6008091E10084FF2BC080917A
:10205000E20084FF27C084E089BD89B5826089BD24
:1020600009B400FEFDCF8091D8008F7D8093D80009
:102070008091E1008F7E8093E1008091E2008F7E6D
:102080008093E2008091E20081608093E200809181
:102090004A01882311F481E001C084E080934C015F
:1020A0000E94B1008091E10083FF23C08091E20093
:1020B00083FF1FC08091E100877F8093E10082E071
:1020C00080934C0110924A018091E1008E7F8093B1
:1020D000E1008091E2008E7F8093E2008091E20037
:1020E00080618093E200D4DD80E060E042E1BDDD0C
:1020F00071DF8091E10082FF0AC08091E20082FFDF
:1021000006C08091E1008B7F8093E10063DFFF9147
:10211000EF91BF91AF919F918F917F916F915F915F
:102120004F913F912F910F900FBE0F901F901895D8
:102130001F9380914C01882361F01091E900109267
:10214000E9008091E80083FF01C06ADC17701093FA
:10215000E9001F9108955527002480FF02C0060E54
:10216000571F660F771F6115710521F096958795AA
:10217000009799F7952F802D0895F999FECF92BD7C
:1021800081BDF89A992780B50895262FF999FECF39
:102190001FBA92BD81BD20BD0FB6F894FA9AF99A84
:0A21A0000FBE01960895F894FFCFDA
:1021AA004156524953505F4D4B32008012018123F0
:1021BA0001900001910101920C01943201980603E9
:1021CA009E0002A10001A400024000410142430313
:0C21DA00C00100011289AB45CDD888FF80
:00000001FF
